:1000000083160130850086018312960197019801BD
:100010009C019F01222982070434013402340234F6
:10002000013404340234043402340134043402341C
:10003000043402340134043404340134013404340B
:1000400002340134023401340434023404340234FE
:1000500002340134043402340434023401340434EC
:10006000043401340134043402340134FF34FF34E5
:10007000FF34FF3482076E343F343E34003438346A
:100080003F346D3479340034FF347834303479348B
:100090000034FF34860186038520E7308600852002
:1000A000C33086008520813086008520860185202A
:1000B000813086008520C33086008520E7308600A9
:1000C000852086018603852086019D0A080064300C
:1000D0009B0000009A0B6928051872281F109B0BC3
:1000E000692808001F186F289F1A78289F167D28F6
:1000F0001F1B7C281F177D289F171F146F280A308D
:1001000090006720900B8128080034309B0000008D
:1001100005188F289A0B87289B0B872808001F1427
:100120000800033090006720900B932808000430EB
:100130009C0000009A0B99289B0B99289C0B9928EE
:1001400008000E0886006720860167200E088600DA
:100150009120860191200E0886007F207F207F203D
:100160007F2086017F209C0A9D0A9D0A0800083096
:100170009E008601672067208603672067209E0B0C
:10018000B928860108003030860010211021033084
:1001900092008601102112083A208600FF300606E0
:1001A00003190800920A10211021C9289201C928B8
:1001B0000A309200C92804309E008601860A860D06
:1001C0000318E4286720DF28860C6720860C031CB0
:1001D000E5289E0BDD28860108009F1FF728121CCA
:1001E000F328980A0D29921C0B29970A0D291F1F25
:1001F0000129121CFD28970A0D2992180B29980A2B
:100200000D299F1E0D2912180B29921C0929980AE5
:100210000D29970A0D29970A980A960A9F01080046
:1002200000009A0B10299B0B1029080006309E0035
:10023000F030860091200F30860091209E0B182907
:10024000860108004A201F1C2229860197200F30B2
:100250009D051C080B209100911F30299C01292924
:10026000111C3429B7203929911C3829DB20392960
:1002700016217F201D080B209200921F41299D010D
:100280003929121C472933308E00A1205229921C93
:100290004D2973308E00A12052296D308E00A1208F
:1002A0001F088600ED2003301606031D292996013C
:1002B0009708031D5E2998080319002817081802DB
:1002C000031D6429D8280028031C6829D628002883
:0402D000C328002817
:00000001FF
